:020000040000FA
:020000000C28CA
:08000800F00F0000F01D0A28B2
:10001000F01140140C1009008316031377308F0081
:1000200083120317073099008312031707309A00D1
:10003000831203179E01831203179F018312031378
:1000400000309700831203130130900083160313CE
:1000500080308100831603130C14831203130B17D3
:10006000831603138701831203138B174014C101F6
:10007000C401C301C201C5010230B7000030B8009D
:100080000130B9004018A820C6010130C70001089E
:10009000CA000230810002308A000310460D84003D
:1000A000203E84004A08800203186F28840A800BCF
:1000B0006F284708870646082A3E84000008082261
:1000C000C80000085122C900460D203E840048089F
:1000D0008007840A00300318013049078000C60AEF
:1000E0000310C70D4608053C031D4D28C60103102B
:1000F000460D8400303E84004A0880020318A02880
:10010000840A800BA0284708870607059430C8009A
:100110004430C900031995284608373E840000087A
:100120000022C80000080422C900460D303E8400A9
:1001300048088007840A003003180130490780000E
:10014000C60A0310C70D4608033C031D7728422842
:1001500001308A00C601C10A411DB6284111C20AF8
:10016000421EB628421207300E05C500450816216A
:10017000C30046082A3E8400460800214307800049
:10018000C60A4608053C031DB9280130B71C0230D9
:0E019000B7000130B91C0230B9004010080061
:100200008207243406292B340C290929441C28345C
:100210002734411C24342B3403300E050319033ECC
:10022000033A00210118F43E0800243482071F29F4
:100230002C2939294629532960296D298229420808
:100240000339C800480D82074414003444100834B0
:100250004410033444100A3442080339C800480DDE
:10026000820744140034441003344410053444100D
:10027000083442080339C800480D8207441000348E
:100280004410003444100734441008344208033941
:10029000C800480D82074410003444100234441052
:1002A00005344410073442080339C800480D82075A
:1002B000441000344410FD34441005344410FB3421
:1002C00042080339C800480D820744100034441026
:1002D0000534441000344410FB3442080739C80088
:1002E000480D820744100034441000344414043490
:1002F0004414043444140234441402344410FB34CF
:100300004410FB3442080739C800480D82074414E2
:1003100000344414003444100A34441003344410AC
:0E0320000834441405344410073444100734E4
:100400008207A734C4348B3482070534033407349D
:10041000820783348534A334DD342F349A341C347A
:10042000B3345F341D34EE34D034C134C234D234EA
:10043000EE3418344D348E34DA342F348F34F734AC
:100440006834E1346134E93477340C34A734473408
:10045000ED3498344734FC34B43470343134F434EB
:10046000BC34863453342434F634CC34A4347E344F
:100470005A3438341834FA34DE34C334AA3492345B
:100480007B34663452343F342D341C340C34FD3408
:10049000EF34E134D534C934BE34B334A9349F3495
:1004A00096348207233421341F341D341C341A340B
:1004B00019341734163415341334123411341034FB
:1004C0000F340E340E340D340C340B340B340A3428
:1004D000093409340834083407340734073406343F
:1004E0000634053405340534043404340434043447
:1004F0000334033403340334033402340234023447
:10050000023402340234023401340134013401343F
:100510000134013401340134013401340134013433
:10052000003400340034003400340034003400342B
:04053000003400345F
:02400E00D438A4
:00000001FF
